:100000000CC024C052C022C021C020C01FC01EC0CE
:1000100078C01CC08097A5AFB80011241FBECFE9DF
:10002000CDBF10E0A0E6B0E0E2EAF3E002C0059048
:100030000D92A237B107D9F710E0A2E7B0E001C0F6
:100040001D92AA37B107E1F756D1A9C1D9CF26EB46
:1000500033E003C0F9013197F1F70197D8F708951C
:1000600096B393FB992790F981E0982780917500CA
:10007000880F892B809375008F7090E00895809190
:1000800074008F5F80937400873010F010927400BA
:10009000089580917400811102C086E003C08091B0
:1000A000740081508093740008951895F894A89571
:1000B00084B7877F84BF81B5886181BD11BC789486
:1000C0001092730003C080E190E0C1DFC9DF892B8B
:1000D000D1F78BB780628BBF82E087BB85B7806228
:1000E00085BF889585B78F7D85BF8BB78F7D8BBF8B
:1000F000F894A89581B5886181BD80E481BD78942C
:1001000008951F920F920FB60F9211241F932F93F1
:100110003F934F935F936F937F938F939F93AF938F
:10012000BF93CF93DF93EF93FF938091740081117E
:1001300003C01092760007C0809176008F3F19F0BF
:100140008F5F809376008CDF20917300892B41F1C3
:100150001092780010927700109279002F3F19F0DA
:100160002F5F2093730080917300863191F480910A
:1001700072008111ACC08DDF809176008A3208F068
:10018000A6C0809174008111A2C084E080937200A7
:100190009EC08A3209F09BC085E18093730097C0AE
:1001A0002150243110F46BDF90C0809174008630B0
:1001B00069F480917700909178000196909378008F
:1001C000809377008A3F954108F063DF349B75C0C8
:1001D0002091610020936000C0916200C093610093
:1001E000909163009093620085B180936300D0E0AA
:1001F000C20FD11DC90FD11DC80FD11DD595C795EF
:10020000D595C79580917400813019F482E790E00C
:1002100002C08CE790E0C817D90730F480917900CC
:100220008F5F8093790013C010927900CD39D1058A
:1002300028F083E087BBC09AC4980DC0CF38D105A1
:1002400030F083E187BB88B3816188BB04C082E161
:1002500087BBC49AC09880917200823028F019BC84
:1002600081508093720029C0813039F583E089BDC7
:1002700085E090E0ECDE19BC88EE93E0E8DEE4E196
:10028000F0E010E0849190E08C179D0708F41F5F68
:10029000319680E0E931F807A9F7C0E0DCE009C059
:1002A000D9BD84E690E0D3DE19BC80E991E0CFDED1
:1002B000CF5FC113F5CF10927200809179008C3B13
:1002C00018F0E7DE10927900369A10927300FF91D1
:1002D000EF91DF91CF91BF91AF919F918F917F91DE
:1002E0006F915F914F913F912F911F910F900FBE92
:1002F0000F901F90189517BA88E088BB85BB82E0E5
:1003000087BB83E28FBD81E083BF81E687B9A29A74
:1003100086EC86B9479A81E28FBD8FEF89BD83E075
:1003200090E095DE19BC81E090E091DE85B7877E94
:10033000806185BFBBDEC0E0809174008C17E1F363
:10034000809174008823A9F0E0917400AC2FB0E094
:10035000AC59BF4FF0E0EC59FF4F9C91808198174A
:1003600041F0E0917400F0E0EC59FF4F8081806231
:100370008FBDE0917400F0E0E559FF4F808189BDA9
:10038000C0917400809174008111D6CF81E090E01B
:100390005EDE809172008111F9CF88DECDCFF894B6
:0203A000FFCF8D
:1003A200AAAAAAAA000101030303010001030C285F
:0203B2007DFFCD
:00000001FF
